:060000000000D3EF08F040
:08000800046ED8CF05F0E0CF33
:1000100006F00001E9CF0CF0EACF07F0E1CF08F0DD
:10002000E2CF09F0D9CF0AF0DACF0BF0F3CF12F01C
:10003000F4CF13F0FACF14F0F5CF15F0F6CF16F099
:10004000F7CF17F000C00EF001C00FF002C010F0A3
:1000500003C011F00E01BDAB31EF00F0C5BB2BEFBB
:1000600002F00EC000F00FC001F010C002F011C08D
:1000700003F00CC0E9FF07C0EAFF078E08C0E1FFEC
:1000800009C0E2FF0AC0D9FF0BC0DAFF12C0F3FFBC
:1000900013C0F4FF14C0FAFF15C0F5FF16C0F6FF39
:1000A00017C0F7FF045006C0E0FF05C0D8FF1000DE
:1000B000BE0FF66E000EF7220900F5501200000088
:1000C00000000000005F00000003000300143E1465
:1000D0003E14242A7F2A124333086661364955228A
:1000E000500005030000001C2241000041221C00BA
:1000F00014083E081408083E0808005030000008A4
:1001000008080808006060000020100804023E5142
:1001100049453E04027F000042615149462241495F
:1001200049361814127F1027454545393E4949493B
:100130003201017109073649494936264949493E84
:100140000036360000005636000008142241001424
:1001500014141414004122140802015109063E41EE
:1001600059555E7E0909097E7F494949363E41411C
:1001700041227F4141413E7F494949417F09090967
:10018000013E4141493A7F0808087F00417F410014
:10019000304040403F7F081422417F404040407F34
:1001A000020C027F7F0204087F3E4141413E7F09ED
:1001B0000909061E2121215E7F0909097626494980
:1001C000493201017F01013F4040403F1F20402054
:1001D0001F7F2010207F41221C2241070870080742
:1001E0006151494543007F4100000204081020008E
:1001F00000417F00040201020440404040400001F1
:1002000002040020545454787F4444443838444411
:100210004444384444447F385454541804047E05FC
:1002200005085454543C7F0804047800447D400081
:100230002040443D007F1028440000417F40007C66
:10024000047804787C0804047838444444387C14E6
:10025000141408081414147C007C08040448545432
:10026000542004043F44443C4040207C1C20402057
:100270001C3C4030403C44281028440C5050503C1A
:100280004464544C44000836414100007F00004162
:100290004136080002010204020020202020202014
:1002A000202020202020202020200000202020208E
:1002B0000000493243204552524F522025782000F9
:1002C0005253534920256C6464426D2020004348FA
:1002D00020534E522025336C6428302D313237297B
:1002E0000000564F4C554D4520004D55544520209B
:1002F0002020200020256C646442202000002D2551
:100300006C64644220200000464D2025326C642E2F
:10031000000025316C64204D487A0000414D2025B5
:10032000346C64206B487A00016A026A006A036ACE
:100330007A5102E1795118E0100E7B6FD89077372F
:100340007837003603367A51035C02E17951005C5C
:1003500007E37951005ED8A003067A51035ED88086
:10036000013602367B2FEAD7120078517A19800BBA
:100370007C6F78AF05D0771F781F772BD8B4782B98
:100380007AAF05D0791F7A1F792BD8B47A2B7751A1
:100390007903F3CF01F0F4CF00F07A03F350002695
:1003A00078517903F3500020026E7CAF05D0011E16
:1003B000021E012AD8B4022A6EEF02F00F015B81FF
:1003C0000000000177910F015BB103D0000177813C
:1003D0000F01000177B109D077910F015BB103D014
:1003E000000177810F01F5D700010F015BB1FED746
:1003F0005FCF02F05ECF01F002C079F001C078F06B
:10040000000178C001F079C002F008EF02F0D6D701
:100410000150362602503722352A3550100806E0A2
:1004200038C001F039C002F014D013D03730396E23
:100430003630386E39323832393238323932383231
:100440000F0E3916376A366A356A38C001F039C07E
:1004500002F0DDEF02F00001676B8DB4672B686B73
:100460008DB6682B2650685D02E0010E276E68C0CD
:1004700026F0255238E0675336E1275234E0276AE8
:100480002B6A2A6A685304E0282AD8B4292A04D09F
:100490002850D8B42906280667C025F02D5222E13D
:1004A0002C5031081FE32C5202E12D521BE0786BD7
:1004B000320E776F2DC07AF02CC079F035DF01C095
:1004C00069F06951040802E2040E696F29C078F0EE
:1004D00028C077F07A6B69C079F047D702C029F05D
:1004E00001C028F00BD067C025F02C502C0803E188
:1004F0002D2C01D003D02C2AD8B42D2A29BE17D0F8
:10050000295203E12850000812E2285029100EE079
:100510002850D8B4290628062150C00803E12250EB
:10052000030803E0212AD8B4222AEFD713D029AE3A
:1005300011D0285029100EE0282AD8B4292A215099
:10054000EE0803E12250020804E02150D8B422064C
:100550002106EFD7676B8DB0672B675325E13C52BF
:1005600002E0010E2E6E3D50F40803E13E2C01D056
:1005700004D03D2AD8B43E2A06D0010E2F6E2C0E90
:100580003D5E010E3E5A3F50B80803E140500B0853
:1005900004E03F2AD8B4402A06D0010E306EBC0ECB
:1005A0003F5E020E405A06D03E6A3D6A406A3F6A8C
:1005B0002F6A306A67C03CF02AD702C024F001C01D
:1005C00023F00E01C59B000131EF00F0EA6A5B0EDB
:1005D000E96EEF500EE0140E016E006A002EFED799
:1005E000012EFBD7BF0E006E002EFED700D0EF2EDF
:1005F000F2D712000F011369000E536F010E0C6F3A
:10060000000E146F1C6F5A513F0B016E5A6B5BAF9B
:1006100006D0015204E05B8100005BB1FED7080EFA
:10062000556F566B5351030BFD0F03E13F0E016EE7
:1006300002D01F0E016E01C052FF100E576F616A8B
:10064000840E5B6F889A838A8888838887948284E3
:1006500087828282000138EF09F0838A050E006EDE
:10066000002EFED783988898050E006E002EFED7C8
:10067000839A050E006E002EFED712008888050EA4
:10068000006E002EFED7838A050E006E002EFED768
:10069000839A050E006E002EFED71200839888986C
:1006A000050E006E002EFED7838A050E006E002E0A
:1006B000FED7839A050E006E002EFED71200646BE3
:1006C0008888050E006E002EFED7838A050E006E08
:1006D000002EFED78DA805D0050E006E002EFED789
:1006E000F9D7839A050E006E002EFED7050E006E18
:1006F000002EFED783988898050E006E002EFED738
:100700006451640804E1010E016E03D002D0000EB2
:10071000016EC5EF03F083988898050E006E002ED9
:10072000FED7838A050E006E002EFED78888050E40
:10073000006E002EFED7120063AF02D09FDF01D003
:10074000ADDF63AD02D09ADF01D0A8DF63AB02D08A
:1007500095DF01D0A3DF63A902D090DF01D09EDF37
:1007600063A702D08BDF01D099DF63A502D086DFBB
:1007700001D094DF63A302D081DF01D08FDF63A1BA
:1007800002D07CDF01D08ADF9AD7015203E0C3DFB9
:10079000010E016E12001B5222E15FDF780E636FC3
:1007A000CBDF636BC9DFAD0E636FC6DF8B0E636F8C
:1007B000C3DFAF0E636FC0DF4D5207E0A10E636F62
:1007C000BBDFC80E636FB8DF06D0A00E636FB4DF67
:1007D000C00E636FB1DF9FDF000E016E26D01B2CB1
:1007E00022D03BDF780E636FA7DF636BA5DF8D0E32
:1007F000636FA2DF140E636F9FDFAF0E636F9CDF2A
:100800004D5207E0A10E636F97DFC80E636F94DF50
:1008100006D0A00E636F90DFC00E636F8DDF7BDFAD
:10082000000E016E02D0010E016E1CEF04F04CC0F0
:100830001BF0010E4D6EAFD740EF09F01B522CE1BB
:100840004E6A4E50070828E308DF780E636F74DFA6
:10085000636B72DF636B70DF100E636F6DDF4E5082
:10086000B0094F6E636F68DF56DFF7DE780E636F97
:1008700063DF400E636F60DF4D6A4C6A4D5209E1E1
:100880004C50830806E3636B57DF4C2AD8B44D2ADB
:10089000F5D741DF4E2AD5D71B2C2FD0DEDE780EC0
:1008A000636F4ADF636B48DF200E636F45DF636B66
:1008B00043DF210E636F40DF636B3EDF7F0E636FAC
:1008C0003BDF220E636F38DF636B36DF070E636F2B
:1008D00033DF21DFC2DE780E636F2EDF400E636FE1
:1008E0002BDF4D6A4C6A4D50030806E3636B24DF2F
:1008F0004C2AD8B44D2AF7D70EDF85EF04F05CC040
:100900001CF05DC01DF0120099D75C6A5D6AF7DFCC
:1009100042EF09F082840F0E006E002EFED700D049
:10092000829287920F0E006E002EFED700D0829426
:100930000F0E006E002EFED700D0120087820F0E21
:10094000006E002EFED700D082840F0E006E002EA7
:10095000FED700D082940F0E006E002EFED700D07E
:100960001200829287920F0E006E002EFED700D0EA
:1009700082840F0E006E002EFED700D082940F0EE0
:10098000006E002EFED700D012005A6A5A50060898
:1009900009E359AE02D0D2DF01D0E3DFD890593657
:1009A0005A2AF4D712005AC05CF05BC05DF0A7DF92
:1009B000120062516403F3CF01F0F4CF00F065033D
:1009C000F350002663516403F3500020026E1200BE
:1009D0005E501F08D8B056D040DE780E636FACDE94
:1009E000636BAADE1D50B009626F636FA5DE1C50F9
:1009F000060DF350020F5F6E5F500F0B626F636F57
:100A00009BDE5F38006E0F0E001600500F0B1009B2
:100A1000626F636F91DE7FDE20DE780E636F8CDEA7
:100A2000400E636F89DE200E5E5C606F616B61510A
:100A300004081BE3636B60C062F0656B050E646FB6
:100A4000B8DF02C063F001C062F061510124016EA1
:100A5000000E0220036E015003C0F7FF58EC00F0B7
:100A6000626F636F69DE612BE2D7636B65DE53DE15
:100A70001C2A1C50150806E11C6A1D2A1D50080876
:100A800001E11D6A47EF05F05DC05EF0A1D71200DD
:100A90000900F6CF5BF0F7CF5CF0F5CF5DF0F4DF47
:100AA0005BC0F6FF5CC0F7FF5A2EF2D712005BBEA8
:100AB0000FD00F0E006E5A3800160A0E005C03E2CB
:100AC000300E002602D05B50002600C05DF0DCDF57
:100AD0000F0E5A160A0E5A5C02E2300E02D05B9ECE
:100AE0005B505A265AC05DF0CFDFB5EF05F0596A6A
:100AF00087820F0E006E002EFED700D082840F0E6C
:100B0000006E002EFED700D08CA20BD00F0E006E10
:100B1000002EFED700D0592A5950640801E101D0B7
:100B2000F3D782940F0E006E002EFED700D00F0E6A
:100B3000006E002EFED700D0829287920F0E006EBC
:100B4000002EFED700D0595064081DE15A6A5B6A36
:100B50002ADFB20EF66E020EF76E0A0E5A6E98DF9C
:100B600020C05AF0570E5B6EA2D7200E5D6E8CDF50
:100B7000040E5A6EFA0E5B6E29DD5A2EFBD7010E5B
:100B8000016E03D002D0000E016E12008292879295
:100B90000F0E006E002EFED700D082840F0E006E66
:100BA000002EFED700D087820F0E006E002EFED7DB
:100BB00000D0120054C020F0ADDE54C059F0E5DE84
:100BC000D0DE95DF015204E0E1DF010E016E4DD071
:100BD000586A5850070809E355AE02D0AFDE01D07D
:100BE000C0DED8905536582AF4D781DF015204E090
:100BF000CDDF010E016E39D0586A5850070810E356
:100C0000000B006E5750800B036E0050031002E083
:100C100095DE01D0A6DED89056365736582AEDD745
:100C200066DF015204E0B2DF010E016E1ED0586A89
:100C30005850070810E3000B006E5750800B036EEE
:100C40000050031002E07ADE01D08BDED8905636D9
:100C50005736582AEDD74BDF015204E097DF010EDB
:100C6000016E03D093DF000E016E12008782828432
:100C70000F0E006E002EFED700D08CA203D0010E06
:100C8000576E01D0576A82940F0E006E002EFED769
:100C900000D057C001F0120052C020F03BDE52C01D
:100CA00059F073DE5EDE23DF015206E06FDF010ED6
:100CB000016E000E026E85D0546A5450070809E395
:100CC00053AE02D03BDE01D04CDED8905336542ACE
:100CD000F4D782840F0E006E002EFED700D08782DC
:100CE0000F0E006E002EFED700D082940F0E006E05
:100CF000002EFED700D082840F0E006E002EFED78D
:100D000000D0829287920F0E006E002EFED700D088
:100D100082940F0E006E002EFED700D052C059F004
:100D200034DE0CDEE4DE015206E030DF010E016E3F
:100D3000000E026E46D0566A556A546A545007082F
:100D400009E3D8905536563691DF015201E05580BF
:100D5000542AF4D7829287920F0E006E002EFED78F
:100D600000D082840F0E006E002EFED700D0829439
:100D70000F0E006E002EFED700D0546A54500708A4
:100D800009E3D8905536563671DF015201E055809F
:100D9000542AF4D787820F0E006E002EFED700D0A3
:100DA00082840F0E006E002EFED700D082940F0EAC
:100DB000006E002EFED700D0E9DE55C001F056C00F
:100DC00002F01200EACF5AF0E9CF59F053AE08D042
:100DD000598E59A8592A521E531E522AD8B4532A42
:100DE0005338F009556E5526E20F566E320F586E85
:100DF00053500F0B562656265826E90F576E572686
:100E0000572652380F0B5726582657365836581E35
:100E1000583652500F0B58265536070E546E0A0E90
:100E200057065826FDE356065726FDE35506562677
:100E3000FDE354065526FDE3EA6A540EE96E070EFB
:100E40005914599CED52591407E159B8EE5259B84A
:100E500003D0200E006E20D0E926000EEA22E950D1
:100E6000580803E1EA5201E1598CEF50006E08E1A5
:100E700059BC06D059B81BD059B602D0200E0BD0A1
:100E800059AE06D02D0E006EED50599C599E04D0DF
:100E900059865998300E0026EACF53F0E9CF52F028
:100EA00000C05DF0F1DD53C0EAFF52C0E9FFEE5033
:100EB00059ACD5D712006A0E526E030E536EECDE9B
:100EC00002C04FF001C04EF04CC05AF04DC05BF074
:100ED0006ADDD8904F324E324E50215C03E14F50C4
:100EE000225C21E0D8902134506E2234516E518E14
:100EF0006A0E546E030E556E51C057F050C056F036
:100F000059DED8902134506E2234516E6A0E546EE0
:100F1000030E556E51C057F050C056F04BDE22C044
:100F20004FF021C04EF0196AF2BE198EF29E4FC0EA
:100F300078F04EC077F07A6B0A0E796F94EC01F07E
:100F400019BEF28E02C051F001C050F0080EF66ECC
:100F5000030EF76E030E5A6E9BDD040EE96E51C050
:100F600053F050C052F02EDF2E0E5D6E8DDD196AEB
:100F7000F2BE198EF29E4FC078F04EC077F07A6BB9
:100F80000A0E796F94EC01F019BEF28E00C050F099
:100F900003C051F0050EE96E03C053F000C052F0DB
:100FA00011DF160EF66E030EF76E040E5A6E70DD2C
:100FB00083EF09F00900F5520CE0F6CF52F0F7CFBD
:100FC00053F0F5CF5DF060DD52C0F6FF53C0F7FF80
:100FD000F1D712006A0E526E0F0E536E5DDE02C024
:100FE0004FF001C04EF01F0E4E164F6A2430516E66
:100FF0002330506E513250325132503251325032D1
:1010000051325032070E511650504E5C03E1515090
:101010004F5C10E051C04FF050C04EF04F50880967
:10102000536E6A0E546E0F0E556E53C057F04EC07D
:1010300056F0C0DD4CC05AF04DC05BF0B4DCE20E9F
:10104000F66E020EF76EB6DF4E5208E14F5206E121
:10105000EA0EF66E020EF76EADDF2FD01F0ED880AF
:101060004E56000E4F56D8904E364F364E5214E123
:101070004F5212E1200E5D6E07DD100EE96E4FC07B
:1010800053F04EC052F09EDEF80EF66E020EF76E72
:10109000040E5A6EFDDC11D02D0E5D6EF5DC100EC7
:1010A000E96E4FC053F04EC052F08CDE020EF66E69
:1010B000030EF76E040E5A6EEBDC87EF09F06A0E32
:1010C000526E120E536EE8DD02C04FF001C04EF0BA
:1010D0004F324E324F324E324F324E321F0E4F167B
:1010E0004E164F6A4FC063F04EC062F0656B030E40
:1010F000646F5FDC02C04FF001C04EF09C0E4E26C4
:10110000FF0E4F224CC05AF04DC05BF04CDCC00EBD
:10111000F66E020EF76E050E5A6EBADC100EE96E10
:101120004FC053F04EC052F04DDEC80EF66E020EA8
:10113000F76E050E5A6EACDC8BEF09F06A0E526E3C
:10114000140E536EA9DD02C04FF001C04EF04F32B5
:101150004E324F324E324F324E324F324E324F328B
:101160004E324F324E32030E4F164E9E4F6A4CC0D7
:101170005AF04DC05BF017DCCE0EF66E020EF76E25
:10118000070E5A6E85DC030EE96E4FC053F04EC059
:1011900052F018DED90EF66E020EF76E070E5A6E7A
:1011A00077DC8FEF09F0F86AF29A078E0E01D86BA0
:1011B000D56BD76B080ED96F600ED36F010E1A6E08
:1011C0001B6E1F6A1E6A256A266A276A296A286AB0
:1011D0002B6A2A6A2D6A2C6A2E6A2F6A306A326A52
:1011E000316A346A336A0F010C6B146B1C6B356BFC
:1011F000366B376B346B316B326B336B306B356AFC
:10120000366A376A386A396A3A6A3B6A010E3C6E56
:101210003D6A3E6A3F6A406A416A426A436A010E19
:10122000446E486A476A0E01D86BD56BD76B030EC4
:10123000D96F600ED36F010E5B6E0001E6EC02F019
:101240000E01D86BD56BD76B050ED96F600ED36FBF
:10125000140E5B6E0001E6EC02F00E01D86BD56B4C
:10126000D76B080ED96F600ED36F0001FAEF02F052
:10127000640E5B6EE6EC02F044C04CF017EF04F035
:1012800084EF04F0246A236A6A0E546E040E556ECD
:10129000E00E576E800E566E8DDCC80E5B6EE6EC6F
:1012A00002F0030E226E220E216ED89021344C6E75
:1012B00022344D6E4D8E6A0E546E030E556E4DC027
:1012C00057F04CC056F076DCD89021344C6E223466
:1012D0004D6E6A0E546E030E556E4DC057F04CC0E5
:1012E00056F068DC800ED46E460ED56ED4A801D0C0
:1012F000D36A070ED26E0E01BD8BC00EF2124C6A7D
:101300004D6A0001D8D54C6A010E4D6E63D64C6A09
:10131000030E4D6ED4D64C6A040E4D6E0FD7020EDE
:101320004C6EC80E5B6EE6EC02F04C2EFAD70E0146
:04133000E6D70300F9
:020000040030CA
:0C0000008CFFFCFF9FFFFFDFFEFFFFFFF7
:00000001FF
